:030000000219FDE5
:03000B000200AA46
:03002B0002015679
:03005B000202DFBF
:030073000202CCBA
:1000800002030406080C10182030406080040608A3
:100090000C10182030406080A0C00003070F1F0D17
:1000A0000D04050D050205030302C2AFC0D0C0E078
:1000B000206214E5256009E473E525F4F58AD2622F
:1000C000D0E0D0D0D2AF3285268AC262E526F46075
:1000D00029D0E0D0D0C290C291C292D2AF32C290A9
:1000E000C291C292206F0C2065097405D5E0FDE530
:1000F0007B4290D0E0D0D0D2AF32758A00C28DD290
:100100006201F301B9306805206502D29001B9306F
:100110006805206502D29101B9306805206502D2D8
:100120009201B9C29330680A2065077432D5E0FDA8
:10013000D29001B9C29430680A2065077432D5E0C4
:10014000FDD29101B9C29530680A2065077432D595
:10015000E0FDD29201B9C2AFC2AD53E6EFC0D0C04C
:10016000E0D2D3D2AFC2CEE52A6007207449152A67
:1001700021B77800790020742EE580307E01F430BC
:10018000E70278FF53DACF207E0343DA20307E0384
:1001900043DA10C2D8C271E580307E01F430E70244
:1001A00079FFC3E89970CB306103752A1820740376
:1001B000752A18885CD27020740DE52B6004152B0D
:1001C00021C743DA01C2D82070024136A85C206101
:1001D00002C2702074367982B70431C3E894F040CB
:1001E0000374F0F8E8C4540F28F87984B703024187
:1001F0000CC313C3138721200802C313200A06C3AC
:10020000C898F8410C28F8500374FFF88822E52DAF
:1002100054066022206B1FE536C333C333F8E56410
:10022000C313C313F9C3952240028922E82522F59E
:100230002250037522FF7882B6044E852224A8241A
:10024000C3E52495614002A861C3E895634002A814
:10025000638825E56670024187C3E8AA669A500361
:10026000E8FAE4F9EAC333FBE568F45B29400D25BD
:1002700067F8E56760021567400B41870AC3E567C9
:100280009A5002056778FF882620CF0AD0E0D0D0A8
:1002900043E610D2AD32C2CF053A7801E52A6005B7
:1002A000307402152AC3E55C94014005755F004176
:1002B000C2756000756900E55F2401F55F50037544
:1002C0005FFFD0E0D0D043E610D2AD32C2AF53E6EC
:1002D0007F7592FA7593FFC260759104D2AF32C2F6
:1002E000AF53E6EFC2ADC0D0C0E0C0F0D2D3D2AFC2
:1002F000A8FBA9FCC2D8307102614653DACF207E38
:100300000343DA10307E0343DA20D271E580307E79
:1003100001F420E702611D88278928A17353DACFF1
:10032000207E0343DA20307E0343DA10C2D8C27144
:10033000307402A15F7800E580307E01F430E7027E
:10034000A15F885CA14753DACF207E0343DA2030D7
:100350007E0343DA10C271206102811F53DACF207D
:100360007E0343DA10307E0343DA20C2D8D271888C
:10037000578958C3E89555F8E99556F97B007E08EA
:100380007A00C3E8948CE994005005755B008111F4
:10039000882178A2E6A8216055C3E894C8E99400B2
:1003A0005008E4D2E4FB7A0A61ECC3E89468E9946B
:1003B000015008E4D2E3FB7A0F61ECC3E894D0E982
:1003C00094025008E4D2E2FB7A1E61ECC3E894A0E8
:1003D000E994055008E4D2E1FB7A3C61ECC3E8946F
:1003E00098E994085008E4D2E0FB7A787E00C3E8EC
:1003F0009559FCE9955AFD30E70AECF42401FCED2F
:10040000F43400FD755B00C3EC9AED9E5003755B00
:10041000018859895A8557558558567802A147C38E
:10042000E89527F8E99528F9307C02A12B307B026A
:10043000A12B307A02A1242075028142E9FDE8FC5B
:100440008161E9C313F9E813F8307902A124E9C303
:1004500013F9E813F8307802A124E9C313FDE81377
:10046000FC20612CC3EC941CED940240028178EDD9
:0E047000701EC3EC94C850180529E5297002CF
:10047E001529C3E529940A5002A15F755C00D2705C
:10048E00A15FE529600215297888E6F97400207FBE
:10049E00087896B90302789EE624FAFEE43400FF4B
:1004AE00C3EC9EFCED9FFD9208B90310A208500705
:1004BE00207609D27681CA307602C276A20850160C
:1004CE00B9030DECF42401FCEDF43400FD0204E458
:1004DE0078007900A12BB90315EC33FCED33FDC385
:1004EE00EC940AFCED9400FD50047C007D00C3ECFE
:1004FE0094FFED9400400678FF7900A12BEC8572F5
:10050E00F0A4C5F0A2F733F879004003020547784E
:10051E00FF7900020547E9C313F9E813F8307C0EA2
:10052E00E9600278FFC3E81338F8E43400F9C3E851
:10053E0094FFE99400400278FF885CD2702061023B
:10054E00A15F741FF4552F4BF52FC274EB7002D2BE
:10055E0074752A18307403752A0A306102A173204B
:10056E00740353DAFE207403752B06D0F0D0E0D05E
:10057E00D0D2AD43E6103279010205A3790302050C
:10058E00A3790A0205A3791E0205A379640205A3C5
:10059E0079C80205A37817E4D5E0FDD8FAD9F6227A
:1005AE007A147B780205CA7A107B8C0205CA7A0D02
:1005BE007BB40205CA7A0B7BC80205CAE573D5E087
:1005CE0001227902E4C294D5E0FDD291D5E0FDC2BC
:1005DE0091D5E0FDD294D5E0FDE920E002D2903035
:1005EE00E002D292E573D5E0FDE920E002C2903040
:1005FE00E002C2927496D5E0FDD9C9EAF8D5E0FDC5
:10060E00D8FBDBB8C29422C37C007D0075F00005D8
:10061E00F0EA33FAEB33FB50F6EB13FBEA13FAC3B3
:10062E00E9FFE8FEE89AF8E99BF95004EFF9EEF8D5
:10063E00B3EC33FCED33FDD5F0DFEDF9ECF822E849
:10064E0089F08A20D2D4F8A9F07B0030F70B7BFF1B
:10065E00F42401F8E9F43400F9E88520F0A4ADF0B3
:10066E00F8E98520F0A4AFF0FEED2EF974003FFA04
:10067E007C04C3EA13FAE913F9E813F8DCF48BF0FF
:10068E0030F70AE8F42401F8E9F43400F9E889F0C7
:10069E00C2D4F8A9F0227882B604030206FFC3E59D
:1006AE005C940140030206C9852224E4F544F54515
:1006BE00F546F547F548C26E0206FF7882E6FCD293
:1006CE006EE522F523783879C7AA40AB41C3EB1308
:1006DE00FBEA13FAEC146013C3EB13FBEA13FAEC08
:1006EE0014146007C3EB13FBEA13FAD1158844897F
:1006FE004522C3E5449523F8E5459400F9500CC313
:10070E00E89480E994FF4016020730C3E8947FE92D
:10071E0094005003020730787F790002073078800A
:10072E0079FF8849894A22E5492546F8E54A354741
:10073E00F9854A20E4300701F43548FA30E709C359
:10074E00EA94F0401502076EC3EA940F50030207B5
:10075E006E78FF79FF7A0F02076E780079007AF0D3
:10076E00C3E5249561500AC374019524500B02070A
:10077E008CE54A20E70E02078CE54A30E7068846EC
:10078E0089478A482278A5E6FAC3E54933F8E54A4F
:10079E0033F9D14DE930E70BC3E89480E994FF407B
:1007AE0013E1C6C3E8947FE994005002E1C6787F56
:1007BE007900E1C6788079FFE820E715C3E5239834
:1007CE00F84009C3E8940140030207ED78010207DF
:1007DE00EDE8F424012523F840030207ED78FF88A5
:1007EE004B2278A6E6FAA847A948D14DE930E70C86
:1007FE00C3E89401E994FF4016020821C3E894FF70
:10080E00E99400500302082178FF7900020821784C
:10081E000179FFE920E715C3E54B98F84009C3E8D5
:10082E00940140030208487801020848E8F42401C4
:10083E00254BF8400302084878FF88242278FF20D1
:10084E00692879A1E76023E541601F74FF8541F0B7
:10085E00848539F0306A0375F005A4F8C5F060029E
:0E086E0078FFC3E895645002A864886322C333
:10087C00E5409440E5419401E563500314018C0478
:10088C006002F563220208942275E890227883E6D0
:10089C00FF30EDF9A8BDA9BE0570C3E57094084002
:1008AC0052757000E9FA79A0E76044EA7007E571C7
:1008BC00601B0208CDC3E895716010E571500660AD
:1008CC000C140208D90460F90208D9E571F571C35A
:1008DC0094F6401B7561C0C394064013756180C3C8
:1008EC009406400B756140C3940640037561007516
:1008FC00BB0022E5612410500274FFF5617982B7C8
:10090C0004022126C3A861E524985002A824C3E858
:10091C0095634002A86388258826E570B4070375A3
:10092C00BB1022743279A787F0A4C5F0A2F733F874
:10093C00C3E895614002A86188228824882588260E
:10094C008864227540007541F022C2AF75C820A89A
:10095C00CCA9CDAA3A30CF010A75C824D2AFAB3B93
:10096C00AC3C883B893CC3E89BF8E99C206908F9BE
:10097C00306602416521BFAD3D8A3DF9EA9DFA60C2
:10098C000478FF79FFAE3EAF3F8B3E8C3FA83BA96E
:10099C003CC3E89EF8E99FF9C3E54113FBE540131E
:1009AC00FAE82AF540E93BF54150067540FF7541E0
:1009BC00FF410CAA40AB41AC40AD417E047F02C369
:1009CC00EB9404400D1E1FC3EB94084005206A02F3
:1009DC001E1FC3ED13FDEC13FCDEF7C3EA9CFAEB10
:1009EC009DFBEF6009C3E913F9E813F8DFF7EA2878
:1009FC00FAEB39FB8A408B4150067BFF8B408B41D5
:100A0C00C3EB94025002D2663069047F03413778FD
:100A1C0092E6FFC3E537948240110FC3E53794A0EB
:100A2C0040010FC3EF940640027F057E02E541C4EE
:100A3C00540FF9E541C454F0F8E540C4540F28F8BC
:100A4C00C3E89EFAE99400FB4009C3EA9402EB94D4
:100A5C000050047A02E4FB41B1AA40AB41EBC4FE66
:100A6C00EAC4540F4EFCC3EA9CFAEB9400FBC3E8B7
:100A7C0013C313F8EA28FAEB3400FB8A408B41C30A
:100A8C00EB94024002C2667802EBC4FE7B00EAC41F
:100A9C00540F4EFAC3EA98FA4005C3940250027AF6
:100AAC00027892E6FF30600241B1855192855293F3
:100ABC00D26043E680C3E49AF8E49BF930660261A5
:100ACC003DE8FAE9FBD3E913FDE813FC88518952A0
:100ADC00C3EF94036038EF20E00DE82CF8E93DF902
:100AEC00ECFAEDFB020B06E828F8E939F9C3E82427
:100AFC0002F8E93400F97AFE7BFFC3EF9403400E51
:100B0C008A538B54884D894E8C4F8D50617188530C
:100B1C0089548A4D8B4E8C4F8D503069127553F021
:100B2C007554FF754FF07550FF7551F07552FF619C
:100B3C0071E8FAD3E813FC8851C3EF94036020EFFB
:100B4C0020E007E82CF8ECFA615DE8282402F87A3A
:100B5C00FEC3EF940340088A53884D8C4F61718813
:100B6C00538A4D8C4FE568C3335002646BF5683083
:100B7C006002617B753402D26043E680E52D540639
:100B8C006034A840A941C3E913F9E813F8C3E91389
:100B9C00F9E813F8306904E92440F9C2AF53E67F51
:100BAC00759100C3E498F594E499F595759104D288
:100BBC006043E680D2AF22D26475430075200030CA
:100BCC006C03752040020BE2D26475430075204023
:100BDC00306C0375200078017901206620E52D54D6
:100BEC00066002C2647914E541C313700104F8C3B2
:100BFC00941440027814306904781B791B2060101F
:100C0C00E543600C306903D53404D26D818D71835A
:100C1C000543E59BF45440B52002817730690908FF
:100C2C00C3E899400118810920640A08C3E8994077
:100C3C000261E28109C264C2AF53E67F7591003054
:100C4C0066127594007595F8759104D26043E68030
:100C5C00D2AF61E2E5417EFFC3334005C3334001AF
:0E0C6C00FEC3E49E759400F5958154C3E533F4
:100C7A009401500261E230640261E2D802818B8100
:100C8A0009C26DC2AF53E67F7591008553948554AE
:100C9A0095759104854D92854E93D26043E680D234
:100CAA00AFE52D54066008206A020533020CC930EC
:100CBA006D0D206C0A2064071581158102157322B7
:100CCA0078003064027801E53775F007A4F9E5F099
:100CDA0028F5F0E9A2F013A2F113A2F213F537C333
:100CEA0094785003753778C3E53795384008D2654C
:100CFA00C290C291C292306002A100854F92855083
:100D0A0093D26043E68022207D16C2AF754202C2AA
:100D1A0094D293306202D292D2AF759F11020F0021
:100D2A00C2AF754202C294D295306202D290D2AF5B
:100D3A00759F11020F00307243207D20C2AF7542A9
:100D4A0003900134757B10C292C295306204D2912D
:100D5A00A15ED294D2AF759F21020F00C2AF754235
:100D6A0003900134757B10C290C293306204D29111
:100D7A00A17ED294D2AF759F01020F00207D17C2C7
:100D8A00AF75420390010FC292306202D291D2AF84
:100D9A00759F21020F00C2AF75420390010FC290E6
:100DAA00306202D291D2AF759F01020F00207D16E8
:100DBA00C2AF754204C293D295306202D291D2AFC9
:100DCA00759F01020F00C2AF754204C295D29330DB
:100DDA006202D291D2AF759F21020F003072432076
:100DEA007D20C2AF754205900123757B08C291C26E
:100DFA0094306204D290C104D293D2AF759F11028B
:100E0A000F00C2AF754205900145757B20C291C2A1
:100E1A0094306204D292C124D295D2AF759F110246
:100E2A000F00207D17C2AF754205900105C29130AF
:100E3A006202D290D2AF759F11020F00C2AF754203
:100E4A0005900119C2913062EBD292D2AF759F110F
:100E5A00020F00207D16C2AF754206C295D29430A9
:100E6A006202D290D2AF759F21020F00C2AF7542C3
:100E7A0006C293D294306202D292D2AF759F010217
:100E8A000F00307243207D20C2AF754201900145A8
:100E9A00757B20C290C293306204D292C1AAD295C5
:100EAA00D2AF759F01020F00C2AF754201900123B4
:100EBA00757B08C292C295306204D290C1CAD2939D
:100ECA00D2AF759F21020F00207D17C2AF75420174
:100EDA00900119C290306202D292D2AF759F01027C
:100EEA000F00C2AF754201900105C292306202D270
:100EFA0090D2AF759F21C26522900103757B00C213
:100F0A0090C291C292C293C294C295C26222788060
:100F1A0076090876090876040876FF0876030876C3
:100F2A00FF08760B087601087601087601788C7638
:100F3A00010876FF0876FF0876FF0876FF0876FF35
:100F4A000876030876FF0876FF0876FF08762508F4
:100F5A0076D00876280876500876040876FF087650
:100F6A000208760008767A0876FF08760108760184
:100F7A00087600087603087600227887E6FFC272B0
:100F8A007888E6C394036008C27DE630E102D27D28
:100F9A00C27E7889E630E102D27EC3EF940260080D
:100FAA00758E01D273020FB7758E00C273227880D4
:100FBA00E6149000809378A5F67881E61490008074
:100FCA009378A6F67886E61490008D9378A7F6783B
:100FDA0086E6F539C394025003753902789CE675A2
:100FEA0038FFB402037538A0B4030375388278A3B6
:100FFA00E61490009A93F566120F0322227896E679
:10100A00FA7897E6FB7888E6B40305C3EB940EFBFF
:10101A00307F047A007BFFC3EB9AFCC394825002B0
:10102A007C827572000572EC8572F0A4C3E5F094B7
:10103A007D40F222D27F11071205941205947A009C
:10104A007B007C1012058AE55C2AFA74003BFBDC03
:10105A00F37C04C3EB13FBEA13FADCF7FEC27F113D
:0D106A000722757C00757D00E5EF20E60390
:101077007520000520903FFFE520146006901DFFB6
:101087001460009304600375EF1453D9BF7581C0D2
:1010970043FF8012058575EF0443B203E5B32402CD
:1010A70020E70DF521E5E320E0068521B343E301C1
:1010B700120F037580FF75A40075F19075D47F75C5
:1010C700903875A53F75F23F75D50075A60175E295
:1010D70041120F03E4F8F6D8FD756801120F1812D4
:1010E70015C478988673753001C2AF12059E120534
:1010F700AE1205941205B51205941205BC1205949B
:10110700C2AF757C00757D0078FA79FA308707D908
:10111700FBD8F7021C00120F84120FB81106110733
:1011270078988673120F0375881075890275C8241D
:1011370075910475D84075A82275B80275E6907543
:101147009B80759D0075D10775BC5875BB0075BA36
:101157001175E880120585D2AF12089175360053D4
:10116700DACF207E0343DA20307E0343DA1043DAF6
:1011770001C2D8C27112059ED2617B037A0CE55B6E
:1011870070077A0CDB030211071205942070030223
:101197001107C270E55CC3940240E1E52F541F8537
:1011A7005E5DF55EB55DD5DAD5C26153DACF207ED7
:1011B7000343DA20307E0343DA10C2D8C27178A223
:1011C700E67008D274E52F54E0F52FC27575290033
:1011D700120599307409C3E529940A4002D27512A1
:1011E700058A78023074027800C3E55C9840F0C243
:1011F700AF1205AE1205AE1205AED2AF12059E753F
:101207004C007888E6B4030241FC12058A788CE624
:10121700C3940150030212FCE530C394015003024A
:1012270012FC757CA5757DF1207435C3E55C94FFD0
:1012370050030212FCC2AF1205C3D2AF120599C305
:10124700E55C940150EFC2AF1205AE12058F12058F
:10125700AED2AF120599C3E55C94FF40E90217705F
:101267007F02D27F1107120599C2AFC27F1107AE65
:101277005CC3E55C947FD2AF5002610C120585C256
:10128700AF1205C3D2AFDFDA113EC3EE7897F6127D
:10129700059E1216F37F0AD27F1107120599C2AF76
:1012A700C27F1107AE5CC3E55C947FD2AF50E612F4
:1012B7000585C2AF1205AE12058F1205AED2AFDF9C
:1012C700D6113EEE24037896F6F87997E7C3948211
:1012D7004003985006E824827897F612059E121666
:1012E700061217221205991107C3E55C94FF5002F5
:1012F7004129021770757C00757D00C3E55C954C2C
:101307004003855C4C12059978017988E7B403029C
:101317007805C3E55C9840024109C2AF1205C312C4
:1013270005C31205C3D2AF12059E753000E4F5312F
:10133700F5320531E531F4703F0532789AE67819D0
:10134700146012783214600D787D14600878FA14EE
:101357006003753200C3E53298401D120F03120572
:1013670085153275310078998673C2AF1205C3D2DD
:10137700AF7898867312059912058FE52A700530A4
:101387007402210778012074027806C3E55C98404F
:10139700A17888E6C394036003120599E52A7003D0
:1013A700021107C2AF120F03E4F522F523F524F566
:1013B70025F526F567D2AF7885E6C333F565E4F5FD
:1013C70044F545F546F547F548F570F52CF52DF547
:1013D7003775700875BB1012058512089530EDFD3D
:1013E700A8BDA9BEE97001F888711208997570083F
:1013F70075BB10120F84C2AF7561FF12092F8522CA
:1014070061852262852263D2AF7522017524017539
:101417002501752601856069756A017888E6B40338
:1014270007C27D307602D27DD268D2697533001249
:101437000E5D120E8C12094F12095612094F12092E
:101447005612094F120BD41206A4120CCA120D1110
:10145700120956120BC3306E0312070020660312DF
:0E146700084B30660312087B120CCA120D40AF
:10147500120956120BD4306E03120735120CCA121C
:101485000DB7120956120BC3306E03120793120CD7
:10149500CA120DE6120956120BD4306E031207F06C
:1014A500120CCA120E5D120956120895120BC312C0
:1014B5000CCA120E8C1208991209563069328564CD
:1014C50061856462856069756A0179187A0CC3E57E
:1014D5003399400FC269D26A8A3585646185646330
:1014E5000214F5C3E55C9401400302144B02157B1D
:1014F500306A1D206C1AE535147006C26AD26B81FC
:101505004BF535C3E55C9401400302144B02157B92
:1015150075360078FA79A4E760027803C3E55F9829
:101525005054307404E52A604D7888E6B4031720DA
:101535007D05207607A14B307602A14B206C07D2A2
:101545006C856461818A78F0306C058564617820EA
:10155500C3E541985002814B306C1BC26CC27D3093
:101565007602D27DD26A753512856461814B053666
:10157500E55C6002A17E753600C2AF120F03788765
:10158500E6FE7602120F847887EEF6E4F522F5235F
:10159500F524F525F526F565752C00752D00D2AFDA
:1015A500120599120F0378A4E66006D290D291D263
:1015B50092307409C3E536940440022107613490E2
:1015C5001A0D7820121648E520B4550CA3121648BA
:1015D500E520B4AA030215E6120F18121606021624
:1015E50005901A0378807B0A121648A308DBF99048
:1015F5001A0F788C7B19121648A308DBF9901A2864
:1016050022C2AF12168B121668901A00740E1216AB
:101615004DA3740712164DA3741512164D901A0397
:1016250078807B0A12164CA308DBF9901A0F788C88
:101635007B1912164CA308DBF912169E12167C9024
:101645001A2822E493F622E6438F01538FFDFFC348
:10165500E583941C400122EF857CB7857DB7F05367
:101665008FFE22438F02438F01857CB7857DB7901E
:101675001A0DF0538FFC22901A0D7455D14D901A06
:101685000E74AAD14D227A3079D07820901A40D1A3
:1016950048E520F709A3DAF7227A3079D0901A4085
:1016A500E7D14D09A3DAF922AB74A875BB0102791C
:1016B50080BB02027981BB03027982BB0402798473
:1016C500BB05027986BB06027992BB07027987BB07
:1016D500080279A3BB0902799CBB0A027988BB0B76
:1016E500027989E8F7227C0512059EDCFB22C2AF50
:1016F5001205AE1205B51205BC1205C312058F12EF
:1017050005AE1205B51205BC1205C312058F1205EB
:10171500AE1205B51205BC1205C3D2AF22C2AF1277
:1017250005C31205BC1205B51205AE12058F1205CB
:10173500C31205BC1205B51205AE12058F1205C3FD
:101745001205BC1205B51205AED2AF22AE74AF7547
:10175500C2AF1205AE1205AE1205AE12058FDEF24E
:101765001205C312058FDFF8D2AF22D1F3D1EBD129
:10177500EB757401757501757600F1517C05AD5CED
:1017850012059EC3ED955C70F5C3E55C9401400AB6
:10179500C3E55C94FF40320217ACD1ADD106D1F35D
:1017A500C2AF75EF14D1EBDCD50576C3E5769403AE
:1017B500500280C6D1EB0575E5741490009F93F82F
:1017C50008C3E57598500280AED1EBD1EB0574C323
:1017D500E574940C5002809C120F18D106C2AF75A7
:0417E500EF14D1EB41
:0319FD0002106C69
:101A00000E0715090904FF03FF0B01010155AA0187
:101A1000FFFFFFFFFF03FFFFFF25D0285004FF0259
:091A2000007AFF0101000300FF40
:101A4000234D445258363248232020202020202085
:101A500023424C48454C4923463333302320202031
:101A60002020202020202020202020202020202076
:101C0000C2AFC2D353D9BF7581C043B20343FF8073
:101C1000752438752503B1DC7529A5752AF175E29F
:101C20004043F18053A47F75D4FFD2877DFA7803B7
:101C300079E67C10752200752300901DE97B0675FE
:101C400024987525013087028145208708D8FBD963
:101C5000F9DCF781B7308708D8FBD9F9DCF781B711
:101C6000B19CE493A3C39A6004DDC381B7DBDBB10D
:101C70008E6002812E7B08E493FAA3B16FDBF87AC1
:101C800030B16F752200752300B18EEAFCEBFDC305
:101C9000ED94FE400EB18E8A278B28ED30E0048A49
:101CA000828B83B18E7AC270D8C3ED94FE601950D6
:101CB000CEBD002BEC600F7520007521FF7529004B
:101CC000752A000200008100A827A9280809D80465
:101CD000D90281DCB192EA89AAF281CE0D81A3C337
:101CE000ED94035053EDA2E092007AC5C3E58294CF
:101CF00000E583941C508A200010438F02438F011B
:101D00008529B7852AB7F0300029A827A92808090E
:101D1000438F01538FFDD804D902A133C3E58394C7
:101D20001C4003A3A11689AAE28529B7852AB7F02A
:101D3000A3A116538FFC817F7AC1BD030CE493A34A
:101D4000FAB153DCF8B14B817F8181AA22AB23B178
:101D50006FEBFAEA6222752608C3E52313F523E543
:101D60002213F52250066323A0632201D526EAB18F
:101D7000DCB1DC75260AEAF4200102D287300102C8
:101D8000C287B1DCC3134002C201D526EB22B19257
:101D9000EAFB208702A192308702A197752608AE40
:101DA00024AF25C3EF13FFEE13FEB1E0B1DCC3EAAD
:101DB000133087024480FA30E703632201C3E5232E
:101DC00013F523E52213F52250066323A0632201B5
:101DD000D526D9E52265236523F52222AE24AF2539
:101DE0000E0FDEFEDFFCD20122424C48656C6934E6
:071DF000373163F3300601F7
:00000001FF
